:10000000831614308500003086008312E4288207AE
:100010003E344134413441343E34003410342034D1
:100020007F3400342734493449344934313422345C
:1000300041344934493436340C34143424347F3454
:1000400004347A3449344934493446343E344934EA
:1000500049344934263440344734483450346034C9
:1000600036344934493449343634323449344934E5
:1000700049343E340034910AA60AA60AA60AA60A02
:10008000A60A911C0800911D080000309100A600EE
:10009000920AA70AA70AA70AA70AA70A921C080099
:1000A000921D080000309200A700930AA80AA80A2F
:1000B000A80AA80AA80A931C0800931D080000308B
:1000C0009300A800940AA90AA90AA90AA90AA90AD8
:1000D000941C0800941D080000309400A900950AA3
:1000E000AA0AAA0AAA0AAA0AAA0A951C0800951D21
:1000F000080000309500AA00080085140000851053
:100100002A08A30005309800230807208600C8208D
:10011000A30A980B8428080085140000851029087C
:10012000A30005309800230807208600C820A30AF2
:10013000980B932808008514000085102808A30058
:1001400005309800230807208600C820A30A980BD2
:10015000A22808008514000085102708A300053098
:100160009800230807208600C820A30A980BB1280E
:1001700008008514000085102608A30005309800AB
:10018000230807208600C820A30A980BC02808006F
:100190009B0BC828003086000510000005140800DD
:1001A00004309B009A0BD2289B0BD228080005191B
:1001B000DA28DF289E1A08009E163B2008009E12AF
:1001C0000800051A002808000030910092009300F2
:1001D00094009500A600A700A800A900AA0060301E
:1001E0009C007D20D7209C0BF12820309C00D02043
:1001F000D7209C0BF72860309C008C20D7209C0BCC
:10020000FD2820309C00D020D7209C0B0329603093
:100210009C009B20D7209C0B092920309C00D020DB
:10022000D7209C0B0F2960309C00AA20D7209C0B64
:10023000152920309C00D020D7209C0B1B29603032
:100240009C00B920D7209C0B2129FF309C00D02096
:0A025000D720E1209C0B2729EF289E
:00000001FF
